:200000000C9427040C94BC190C9495190C944F040C944F040C944F040C944F040C944F0493
:200020000C944F040C944F040C944F040C944F040C944F040C944F040C944F040C944F0428
:200040000C944B190C944F040C944F040C944F040C944F040C944F040C944F040C944F04F7
:200060000C94E3190C944F0400407A10F35A00A0724E18090010A5D4E80000E8764817002B
:2000800000E40B54020000CA9A3B000000E1F505000080969800000040420F000000A0863C
:2000A00001000000102700000000E803000000006400000000000A000000000001000000AE
:2000C00000002C76D888DC674F0823DFC1DFAE59E1B1B796E5E3E453C63AE651997696E839
:2000E000E6C28426EB898C9B62ED407C6FFCEFBC9C9F40F2BAA56FA5F490055A2AF75C931F
:200100006B6CF9676DC11BFCE0E40D47FEF520E6B500D0ED902E0300943577050080841EB8
:20012000080000204E0A000000C80C333333330F986E12831141EF8D2114893BE65516CF0E
:20014000FEE6DB18D1844B381BF77C1D901DA4BBE424203284725E228100C9F124ECA1E598
:200160003D27413530560041203556002035305600203230560020313056002020355600DE
:2001800020203256002020315600302E355600302E3256003230306D73003130306D73001E
:2001A0002035306D73002032306D73002031306D73002020356D73002020326D7300202030
:2001C000316D73003530307573003230307573003130307573002035307573006201670166
:2001E0006C01710176017B01800185018A018F0194019A01A001A601AC01B201B801BE01BB
:20020000C401CA01D001D601CDCC4C3ECDCCCC3DCDCC4C3D0AD7A33C0AD7233C0AD7A33B00
:200220006F12033B6F12833A6F12033A17B7513917B7513917B7513900000000003E5B4F13
:200240005B3E3E6B4F6B3E1C3E7C3E1C183C7E3C181C577D571C1C5E7F5E1C00183C1800CC
:20026000FFE7C3E7FF0018241800FFE7DBE7FF30483A060E2629792926407F050507407F88
:2002800005253F5A3CE73C5A7F3E1C1C08081C1C3E7F14227F22145F5F005F5F06097F01F2
:2002A0007F006689956A606060606094A2FFA29408047E040810207E201008082A1C0808AC
:2002C0001C2A08081E101010100C1E0C1E0C30383E3830060E3E0E06000000000000005F37
:2002E00000000007000700147F147F14242A7F2A1223130864623649562050000807030052
:20030000001C2241000041221C002A1C7F1C2A08083E08080080703000080808080800002E
:2003200060600020100804023E5149453E00427F400072494949462141494D331814127FE8
:200340001027454545393C4A49493141211109073649494936464949291E00001400000018
:200360004034000000081422411414141414004122140802015909063E415D594E7C12111A
:20038000127C7F494949363E414141227F4141413E7F494949417F090909013E41415173E2
:2003A0007F0808087F00417F41002040413F017F081422417F404040407F021C027F7F0427
:2003C00008107F3E4141413E7F090909063E4151215E7F09192946264949493203017F0191
:2003E000033F4040403F1F2040201F3F4038403F631408146303047804036159494D4300B9
:200400007F4141410204081020004141417F040201020440404040400003070800205454F3
:2004200078407F284444383844444428384444287F385454541800087E090218A4A49C78B9
:200440007F0804047800447D40002040403D007F1028440000417F40007C047804787C08C4
:200460000404783844444438FC1824241818242418FC7C08040408485454542404043F4451
:20048000243C4040207C1C2040201C3C4030403C44281028444C9090907C4464544C440014
:2004A000083641000000770000004136080002010204023C2623263C1EA1A161123A404048
:2004C000207A385454555921555579412254547842215554784020545579400C1E527212E7
:2004E0003955555559395454545939555454580000457C410002457D420001457C407D12B6
:2005000011127DF0282528F07C545545002054547C547C0A097F4932494949323A44444448
:200520003A324A4848303A4141217A3A42402078009DA0A07D3D4242423D3D4040403D3C8A
:2005400024FF2424487E4943662B2FFC2F2BFF0929F620C0887E09032054547941000044E9
:200560007D413048484A32384040227A007A0A0A727D0D19317D2629292F28262929292646
:2005800030484D4020380808080808080808382F10C8ACBA2F102834FA00007B00000814ED
:2005A0002A142222142A14085500550055AA55AA55AAFF55FF55FF000000FF00101010FFE3
:2005C00000141414FF001010FF00FF1010F010F0141414FC001414F700FF0000FF00FF144A
:2005E00014F404FC141417101F10101F101F1414141F00101010F0000000001F101010103D
:200600001F10101010F010000000FF101010101010101010FF10000000FF140000FF00FFCC
:2006200000001F10170000FC04F414141710171414F404F40000FF00F71414141414141484
:20064000F700F7141414171410101F101F141414F4141010F010F000001F101F0000001F16
:2006600014000000FC140000F010F01010FF10FF141414FF141010101F00000000F010FF9B
:20068000FFFFFFFFF0F0F0F0F0FFFFFF0000000000FFFF0F0F0F0F0F3844443844FC4A4A9C
:2006A0004A347E02020606027E027E0263554941633844443C04407E201E2006027E0202E1
:2006C00099A5E7A5991C2A492A1C4C7201724C304A4D4D303048784830BC625A463D3E4937
:2006E0004949007E0101017E2A2A2A2A2A44445F444440514A444040444A51400000FF016A
:2007000003E080FF000008086B6B083612362436060F090F060000181800000010100030FE
:2007200040FF0101001F01011E00191D1712003C3C3C3C00000000000000000023002600A1
:200740002900000000080002010000030407000000000000000000000000240027002A00E2
:20076000010204081020408001020408102001020408102000000000250028002B0004047C
:2007800004040404040402020202020203030303030356004261747465727920766F6C740D
:2007A000616765005670700056726D730041432044564D2035562072616E67650056004431
:2007C000432044564D2035562072616E6765005670700056726D730041432044564D203539
:2007E00030562072616E676500560044432044564D203530562072616E6765004476616CD3
:200800006C6579456C656374726F6E69637300506F6F72204D616E27732050656E53636F35
:2008200070650025006B48006B4800487A00487A00756E53796E63005600726D0061760048
:20084000414300444300486F6C640000021B11241FBECFEFD8E0DEBFCDBF15E0A0E0B1E032
:20086000EAE8FCE502C005900D92AE36B107D9F728E0AEE6B5E001C01D92A633B207E1F758
:2008800014E0C7E2D4E004C02197FE010E94152EC632D107C9F70E943F1B0C94432E0C946A
:2008A000000028E030E040E8E0912C08F0912D08508190913308909595239083E0912A08DD
:2008C000F0912B0890913208582F542389F05081952B9083E0912C08F0912D0890815091A1
:2008E0003308952B9083469521503109E9F60895508190959523EDCF83B1982F97709730B5
:2009000049F028E833E130936F0520936E0591E09093EA0580FD15C02091A6073091A7077B
:200920002F5F3F4F3093A7072093A6072091A6073091A7072330310524F01092A70710926E
:20094000A60781FD46C02091A6073091A707232BB9F42091A4073091A5072F5F3F4F3093F6
:20096000A5072093A4072091A4073091A5072A30310534F029E030E03093A5072093A4070A
:200980002091A6073091A70721303105B9F420918107309182072F5F3F4F309382072093B8
:2009A000810720918107309182072C30310534F02BE030E030938207209381072091A60776
:2009C0003091A7072230310521F410929D0710929C0782FD45C02091A6073091A707232BE1
:2009E000B9F42091A4073091A507215031093093A5072093A4072091A4073091A5072230EE
:200A0000310534F422E030E03093A5072093A4072091A6073091A70721303105A1F42091FF
:200A2000810730918207215031093093820720938107209181073091820737FF04C0109293
:200A40008207109281072091A6073091A7072230310531F421E030E030939D0720939C079B
:200A600083FD06C08091AA0791E089278093AA07089508950895AF92BF92CF92DF92EF92CD
:200A8000FF920F931F93CF93DF936C017B018B01040F151FEB015E01AE18BF08C017D1075A
:200AA00059F06991D601ED91FC910190F081E02DC6010995892B79F7C501DF91CF911F9133
:200AC0000F91FF90EF90DF90CF90BF90AF900895833081F028F4813099F08230A9F008950D
:200AE0008730A9F08830C9F08430B1F4809180008F7D03C0809180008F77809380000895B5
:200B000084B58F7784BD089584B58F7DFBCF8091B0008F778093B00008958091B0008F7DB5
:200B2000F9CFCF93DF93282F30E0F901EE5BF84F8491F901E05AF84FD491F901E258F84FB8
:200B4000C491CC23A1F081110E946805EC2FF0E0EE0FFF1FE85CF84FA591B491EC91ED2386
:200B600081E090E009F480E0DF91CF91089580E090E0FACF1F93CF93DF93282F30E0F9015A
:200B8000EE5BF84F8491F901E05AF84FD491F901E258F84FC491CC23A9F0162F81110E94FF
:200BA0006805EC2FF0E0EE0FFF1FEC58F84FA591B4918FB7F894EC91111108C0D095DE231D
:200BC000DC938FBFDF91CF911F910895DE2BF8CFCF93DF9390E0FC01E05AF84F249182581A
:200BE000984FFC0184918823C9F090E0880F991FFC01EA5AF84FA591B491FC01EC58F84F4E
:200C0000C591D49161110DC09FB7F8948C91209582238C938881282328839FBFDF91CF9135
:200C20000895623051F49FB7F8943C91822F809583238C93E8812E2BEFCF8FB7F894EC9137
:200C40002E2B2C938FBFEACF61E08CE00E94E80560E08CE00C94BA052091000190E4299F40
:200C600090011124822B80937C0080917A00806480937A0080917A0086FDFCCF8091780014
:200C80009091790008953FB7F8948091D9059091DA05A091DB05B091DC0526B5A89B05C096
:200CA0002F3F19F00196A11DB11D3FBFBA2FA92F982F8827BC01CD01620F711D811D911D8F
:200CC00042E0660F771F881F991F4A95D1F708958F929F92AF92BF92CF92DF92EF92FF927C
:200CE0004B015C010E9443066B017C010E9443066C197D098E099F09683E734081059105CD
:200D0000A8F321E0821A9108A108B10888EEC80E83E0D81EE11CF11C81149104A104B1046D
:200D200029F7FF90EF90DF90CF90BF90AF909F908F90089508950F931F93CF93DF93EC018C
:200D40008E89823009F453C0833009F4ACC0813009F05CC0EC81FD81E41BF50BAF01421BE1
:200D6000530B77FD3FC08E819F8168177907D4F557FF04C0240F351F50E040E08C819D818F
:200D8000FA01E20FF31F8E179F071CF49C01241B350B1216130634F5FB0177FD3796A3E0B4
:200DA000F595E795AA95E1F7F695FE2FEE27F795E795E40FF51FE05FFE4F6770772781E0D8
:200DC00090E001C0880F6A95EAF7482F0130110509F472C008F47CC02E0F3F1F0230110563
:200DE00009F483C0DF91CF911F910F910895AC81BD81CD01861B970BBC0161507109EE8123
:200E0000FF81E41BF50BAF01421B530B77FDEACF8C819D81681779072CF757FF04C0240F21
:200E2000351F50E040E08E819F81FA01E20FF31F8E179F071CF49C01241B350B1216130629
:200E40008CF6922FA42FA695A695A69580E8A89FD0011124A60FB71FA05FBE4F477009F4CB
:200E600057C058E0541B452F652F70E0FB01E85EFA4F8081251708F0B0C0621B71092FEF17
:200E800030E002C0359527956A95E2F7822301301105A9F108F464C00230110509F0A2CFCA
:200EA0002C9182272EC0AE81BF81CD01861B970BBC016150710955CF2E0F3F1FE217F307C4
:200EC00009F490CF8191DF011197842B8C93F6CF80952E0F3F1FE217F30709F483CF919175
:200EE000DF01119798239C93F6CFE217F30709F479CF8191DF01119784278C93F6CF2C919D
:200F0000822B8C93941708F46DCF941BA058BF4F983008F447C00230110531F5FD01892F7E
:200F2000208120952083E058FF4F88508830C0F728EF290F26952695269530E02F5F3F4F3F
:200F40003695322F222737952795A20FB31F977009F448CFE92FF0E0E05FFA4F808132C093
:200F600080952C918223CDCF81E00130110509F080E08195FD01292F8083E058FF4F2850F0
:200F80002830D0F728EF290F26952695269530E02F5F3F4F3695322F222737952795A20FD8
:200FA000B31F9770992309F41DCFE92FF0E0E05FFA4F80810130110541F058F0023011053A
:200FC00009F010CF9C91892702C09C91892B8C9309CF80959C918923FACF0130110509F4C7
:200FE0008ECF08F4BDCF0230110509F459CF8DCF0F931F93CF93DF93EC018E89823009F468
:201000005EC0833009F4B5C0813009F067C0AC81BD81CD01841B950BAC014150510957FD58
:2010200049C08C819D81481759070CF043C077FF04C0260F371F70E060E08E819F81FB013E
:20104000E20FF31F8E179F071CF49C01261B370B121613067CF5922FA62FA695A695A69519
:2010600080E8A89FD0011124A40FB51FA05FBE4F677009F48FC048E0461B642F70E0FB019D
:20108000E85EFA4F8081241708F002C1621B71092FEF30E002C0359527956A95E2F78223E0
:2010A0000130110509F46DC008F49CC00230110509F4F8C0DF91CF911F910F910895EC8140
:2010C000FD81E61BF70BAE81BF81CD01841B950BAC0141505109BF01621B730B57FDEACFB3
:2010E0008E819F81481759072CF777FF04C0260F371F70E060E08C819D81FB01E20FF31F60
:201100008E179F071CF49C01261B370B121613068CF6FA0157FD379693E0F595E7959A95CD
:20112000E1F7F695FE2FEE27F795E795E60FF71FE05FFE4F4770552781E090E001C0880F0F
:201140004A95EAF7482F0130110509F488C008F492C02E0F3F1F0230110509F0ABCFE2172F
:20116000F30709F4A7CF8191DF01119784278C93F6CFEE81FF81E61BF70BBF01621B730B2C
:201180004ECF2C91822B8C93941708F493CF941BA058BF4F983008F447C00230110531F5B2
:2011A000FD01892F208120952083E058FF4F88508830C0F728EF290F26952695269530E023
:2011C0002F5F3F4F3695322F222737952795A20FB31F977009F46ECFE92FF0E0E05FFA4FC2
:2011E000808132C080952C918223CDCF81E00130110509F080E08195FD01292F8083E05841
:20120000FF4F28502830D0F728EF290F26952695269530E02F5F3F4F3695322F22273795FC
:201220002795A20FB31F9770992309F443CFE92FF0E0E05FFA4F80810130110541F058F06C
:201240000230110509F036CF9C91892702C09C91892B8C932FCF80959C918923FACF2E0FB7
:201260003F1FE217F30709F425CF8191DF011197842B8C93F6CF80952E0F3F1F2E173F07C4
:2012800009F418CF9191DF01119798239C93F6CF0130110509F475CF08F4A4CF02301105D2
:2012A00009F075CF2C9182276ECFDC0177FD67C018968D919C911997681779070CF05FC013
:2012C00057FD5DC01A968D919C911B97481759070CF055C056968C9156978230B9F083301C
:2012E00041F1813049F414968D919C91841B950BAB01BC01615071092130310521F108F471
:201300003FC02230310509F458C008951496ED91FC911597E61BF70BBF0161507109169699
:201320008D919C91FC01E41BF50BAF0141505109E3CF16968D919C91861B970BBA01AC0177
:2013400041505109D9CFFA0157FD3796A3E0F595E795AA95E1F7F695FE2FEE27F795E79569
:20136000E60FF71FE05FFE4F4770552721E030E001C0220F4A95EAF78081822B8083089592
:20138000FA0157FD379623E0F595E7952A95E1F7F695FE2FEE27F795E795E60FF71FE05F72
:2013A000FE4F4770552781E090E001C0880F4A95EAF7809590818923E1CFFA0157FD379626
:2013C00083E0F595E7958A95E1F7F695FE2FEE27F795E795E60FF71FE05FFE4F477055270E
:2013E00021E030E001C0220F4A95EAF780818227C5CF0895FC016370668B848195812681CC
:201400003781613039F0633029F091878087338722870895318720879387828708952F92AF
:201420003F924F925F926F927F928F929F92AF92BF92CF92DF92EF92FF920F931F93CF9379
:20144000DF93CDB7DEB76A970FB6F894DEBF0FBECDBF9A8F898F7A8369834A01D22E1887A5
:201460000F833701BC2CDC0159962D913C915A972115310509F015C118968D919C9119978E
:20148000681779070CF0D7C11A968D919C91481759070CF0D0C14C2C512CB6E0CB9E600D11
:2014A000711D11247C876B87161617060CF0C3C1EA2DF0E0FA87E98793E0EE0FFF1F9A9516
:2014C000E1F7F88BEF87CF01840F951F181619060CF0B1C1A98DBA8D58968C91811104C08B
:2014E000BFEABD1508F4D394A98DBA8DED91FC9111970284F385E02DCD010995B5E0DB9E59
:20150000C0011124E981FA81FC83EB83312C212C9C01285C3D4F388F2F8B4A2D50E05E8B9B
:201520004D8BEF89F88DE20DF31D44919E828D82D12CC12C69817A81620D731D7A8B698B0C
:20154000842F90E09C8B8B8BE98DFA8DA081B18140FF82C0F1E0BF126FC0AF126DC01C96E9
:20156000ED91FC912F813885A4014C0D5D1D69897A89898D9A8D0995EB89FC89F595E795AC
:201580004E2F5FEFC51AD50A6D817E818D899E89680F791F7E836D8398E0C916D10481F6F5
:2015A000AFEF2A1A3A0AEB81FC81E40DF51DFC83EB83F5E02F16310409F0B3CF2F813885F5
:2015C00026153705B9F0A98DBA8DED91FC91B1E0BB1257C0AB1255C069817A816B5F7F4F9F
:2015E0000088F189E02D830128E030E0A401898D9A8D0995A98DBA8DED91FC911197068802
:20160000F789E02DCD016A960FB6F894DEBF0FBECDBFDF91CF911F910F91FF90EF90DF908B
:20162000CF90BF90AF909F908F907F906F905F904F903F902F9009941E96ED91FC91EF803A
:20164000F88409851A8592014D815E816B817C81898D9A8D099590CF2F813885261537059A
:2016600009F48ACF31E0B31207C0A31205C01C96ED91FC91930178CF1E96ED91FC91730132
:20168000E0CF6B857C85641975090684F785E02D73010F8518899201A401898D9A8D0995E0
:2016A000A9CFF90134969491329745915491D91AB7E0DB9E400D511D1124F90125913491DD
:2016C0003C8B2B8BFA0125903490FA013296749031963491398B329664903196449041E08A
:2016E0004C1518F04A1508F07FC0662D062C000C770B7C836B83842D042C000C990B9E83F9
:201700008D83A98DBA8DED91FC9111970284F385E02DCD010995512CD12CC12CEA2DF0E0C4
:20172000FA87E9872B2D30E03C872B87A401440D511D47FC5A95588F4F8B69817A81660D2C
:20174000711D67FC7A957E876D877989C71608F051CF2C2D30E04D815E81420F531FA98592
:20176000BA854A9FC0014B9F900D5A9F900D1124FC01E80DF91DF88BEF87852D612C4F8916
:20178000588D420F531F5E8B4D8B671408F050C044244394480E877041F4C1010196EB89CF
:2017A000FC89E20DF31DD4901C01D7FE19C0A98DBA8DED91FC91662D70E0B1E0BB1219C0D4
:2017C000AB1217C02D853E85620F731F0484F585E02D2F8138854D895E89898D9A8D0995E9
:2017E000DD0C6394842DD1CF1E821D821C821B8288CF4B815C81640F751FAB85BC856A9FBD
:20180000C0016B9F900D7A9F900D112469817A81680F791F0684F785E02DEF80F8840985F5
:201820001A859D014F855889898D9A8D0995D8CF570CC3948ACF6A960FB6F894DEBF0FBE66
:20184000CDBFDF91CF911F910F91FF90EF90DF90CF90BF90AF909F908F907F906F905F9027
:201860004F903F902F9008958F929F92AF92CF92EF92FF920F931F93CF93DF93EC01262FEE
:20188000898D9A8D009709F051C06A30D1F41D861C868D8948E0849F900111248E859F8568
:2018A000820F931F9F878E8781E090E0DF91CF911F910F91FF90EF90CF90AF909F908F90BF
:2018C00008956D3089F3CC88AD888F898823C1F08C859D8536E0C39E800D911D112448856E
:2018E00059854817590764F44E855F851D861C8638E0A39EC0011124840F951F9F878E8726
:20190000EA88FB88088919894E855F856C857D85CE010E940F0A2C898C859D8546E0249F9A
:20192000800D911D11249D878C87BECF6A3069F41D861C86FC013896E4912D898E859F850A
:20194000E29F800D911D1124ADCF6D3009F4ACCFFC0134963491631708F4A6CF3296E49151
:20196000E61708F4A1CFFC01329685909490462F431B342F47E0349F800C911C1124F4016D
:20198000329634913196E4913323A9F1EE2399F1CC88F4013596E491AD884F89442301F104
:2019A0000E2E000CFF0BE30FF11DCE9EA001CF9E500D11246C857D85460F571F6885798520
:2019C000641775076CF44E855F851D861C86FC013896E491AE9E400D511D11245F874E877D
:2019E000EA88FB88088919894E855F856C857D85CE010E940F0AF4013496E4912C898C8591
:201A00009D85E29F800D911D11248DCF0F931F93CF93DF938C01D0E0C0E0F801EC0FFD1F42
:201A20006491662341F087E098E00E94340C892B11F02196F2CFCE01DF91CF911F910F911A
:201A40000895682F87E098E00C94340C6F927F928F929F92AF92BF92CF92DF92EF92FF92B9
:201A60000F931F93CF93DF93EC016B015A0139014801E881F9810284F385E02D0995E88112
:201A8000F9810288F389E02D87019301A501B601CE010995A501480D591D41505109E8810E
:201AA000F9810288F389E02D9301B601CE010995E881F9810088F189E02D9401A501B601FD
:201AC000CE010995C60CD71CB60161507109E881F9810088F189E02D9401A501CE01099558
:201AE000E881F9810688F789E02DCE01DF91CF911F910F91FF90EF90DF90CF90BF90AF908F
:201B00009F908F907F906F9009946F927F928F929F92AF92BF92CF92DF92EF92FF920F9350
:201B20001F93CF93DF935C01EB016A01490138018701DC01ED91FC916217730719F56416FD
:201B400075062CF0962D872D3A01C92ED82E9601261937092F5F3F4F048CF58DE02DA3014A
:201B6000BE01C5010995DF91CF911F910F91FF90EF90DF90CF90BF90AF909F908F907F905B
:201B80006F9008954615570591F42617370724F0892D4B01C22FD82F9E01281939092F5F34
:201BA0003F4F068CF78DE02DA601B401DACF0284F385E02D0995D501ED91FC910488F589DB
:201BC000E02D83019401A601BE01C5010995D501ED91FC910688F789E02DC501DF91CF9183
:201BE0001F910F91FF90EF90DF90CF90BF90AF909F908F907F906F900994EF92FF920F937E
:201C00001F93DC011A960D911C911B9718962D913C911997ED91FC9100A0F1A1E02D7B01D9
:201C200050E040E070E060E009951F910F91FF90EF9008954F925F926F927F928F929F92F5
:201C4000AF92BF92CF92DF92EF92FF920F931F93CF93DF936C012B015A0139014801DC0192
:201C6000ED91FC910284F385E02D0995E201640C751CD601ED91FC91C615D7055CF400885B
:201C8000F189E02D87019401A501BE01C60109952196EFCF0688F789E02DC601DF91CF91AF
:201CA0001F910F91FF90EF90DF90CF90BF90AF909F908F907F906F905F904F9009948F9282
:201CC0009F92AF92BF92CF92DF92EF92FF920F931F93CF93DF93EC015B014A016901E881CE
:201CE000F9810284F385E02D099595012C0D3D1D21503109E881F9810488F589E02D78017A
:201D00008401A401B501CE010995E881F9810688F789E02DCE01DF91CF911F910F91FF90FA
:201D2000EF90DF90CF90BF90AF909F908F9009948F929F92AF92BF92CF92DF92EF92FF9215
:201D40000F931F93CF93DF93EC015B014A0169017801E881F9810284F385E02D0995C80C84
:201D6000D91C860101501109E881F9810488F589E02D9501A401B501CE010995E881F98141
:201D80000688F789E02DCE01DF91CF911F910F91FF90EF90DF90CF90BF90AF909F908F9081
:201DA00009940895EF92FF920F931F93DC01ED91FC9100A0F1A1E02D09951F910F91FF90DF
:201DC000EF9008950F931F93DC01ED91FC91068CF78DE02D09951F910F9108950F931F93A9
:201DE000DC01ED91FC91048CF58DE02D09951F910F910895DC01ED91FC910084F185E02D62
:201E000009942F923F924F925F926F927F928F929F92AF92BF92CF92DF92EF92FF920F9345
:201E20001F93CF93DF9300D000D000D0CDB7DEB73C016A013E832D83FC82EB825801A41A78
:201E4000B50AB7FE03C0B194A194B1088D809E80861A970A97FE03C09194819491088A14E3
:201E60009B045CF0902F812F0D811E819D838E839C2D8D2D6B01692F782F0C151D055CF0ED
:201E80009D818E817E836D83692F782F902F812F8601C92ED82E1601201A310A2B012D818C
:201EA0003E81421A530A57FE03C0519441945108710137FE03C03FEFE31AF30AF594E794E9
:201EC0008D819E81861797075CF5A1E0B0E0BA83A983C016D1064CF1D301ED91FC9104847E
:201EE000F585E02D2B813C81A8016D817E818A149B041CF04D815E81B801C3010995E4184F
:201F0000F508F7FE0AC02D813E8189819A81280F391F3E832D83E20CF31C0F5F1F4FD9CFF2
:201F20002FEF3FEF3A832983D4CF26960FB6F894DEBF0FBECDBFDF91CF911F910F91FF9097
:201F4000EF90DF90CF90BF90AF909F908F907F906F905F904F903F902F9008950895209103
:201F6000B105260F3327331F21323105ECF42091D107FC0190E080E0243069F082E008955F
:201F8000A091B1052191AC014F565A4FA40FB52FB11D2C930196861798F38091B105680F8C
:201FA0006093B10580E0089581E008951092D10781E08093D0071092AB0761E082E10E941E
:201FC000BA0561E083E10E94BA05E9EBF0E080818E7F808380818D7F808388E48093B80040
:201FE00085E48093BC000895CF93DF9391E0909390058823B9F0C091B800D091BA00809186
:20200000BC008A7B8093BC0060E082E10E94BA0560E083E10E94BA050E94D60FD093BA0083
:20202000C093B800DF91CF910895CF92DF92EF92FF920F931F93CF93DF93D091FA0781E059
:20204000D13208F09CC0C091F9070E9443066B017C018091D10781116CC082E08093D10710
:2020600081E08093D0078FEF8093CF071092CE07D093CD07A9EDB7E0EDEAF7E080E0D813DA
:202080008DC01092AC078091AC07CC0FC82BC093AC078091AB07813009F084C01092AB0701
:2020A0000E9443066B017C018091AC078093BB008091D3079091D407A091D507B091D607A8
:2020C000892B8A2B8B2BA1F00E9443060091D3071091D4072091D5073091D6076C197D0948
:2020E0008E099F09061717072807390708F442C08091BC0083FDD8CF85EC8093BC000E9423
:2021000043066B017C018091D107823009F44CC08091CF078F3F09F469C08091CF07803275
:2021200009F466C08091CF07803309F463C084E026C08091D3079091D407A091D507B09143
:20214000D607892B8A2B8B2B09F483CF0E9443060091D3071091D4072091D5073091D60737
:202160006C197D098E099F09061717072807390708F06FCF8091D2070E94F40F85E010929F
:20218000D8071092FA071092D707DF91CF911F910F91FF90EF90DF90CF9008959D91919352
:2021A0008F5F6DCF85EEA9CF8091D3079091D407A091D507B091D607892B8A2B8B2B09F4DC
:2021C000A2CF0E9443060091D3071091D4072091D5073091D6076C197D098E099F0906172A
:2021E00017072807390708F08ECFC4CF80E0C7CF82E0C5CF83E0C3CFE091E2058091E1053A
:20220000E81730F4F0E0E059FA4F808190E008958FEF9FEF08959091E2058091E1052FEF75
:202220003FEF981748F4E92FF0E0E059FA4F208130E09F5F9093E205C90108958091E10504
:202240009091E205891B990B0895CF92DF92EF92FF920F931F93CF93DF937C01CB018A01B1
:202260002091D707222389F0EB016B01C40ED51ECC15DD0569F06991D701ED91FC9101906A
:20228000F081E02DC7010995F3CF642F0E94AF0FC801DF91CF911F910F91FF90EF90DF903F
:2022A000CF900895CF93DF931F92CDB7DEB769832091D7072223F9F02091FA07203258F08F
:2022C00021E030E0FC013383228390E080E00F90DF91CF9108958091D807E82FF0E0E752A9
:2022E000F84F998190838F5F8093D8078093FA0781E090E0ECCF61E0CE0101960E94AF0FE3
:20230000F7CFCF93C82F809124088F3FB1F1E0912E08F0912F08808190913408892B80837D
:20232000E0913008F0913108908180913508809589238083E0912E08F0912F089081809196
:20234000340880958923808380912908882389F0CEBD00000DB407FEFDCF8EB5E0912E0810
:20236000F0912F08808190913408892B8083CF9108958C2F0E945104F1CF8091220891E075
:202380009093D7078093F9071092D8071092FA0760E08BEF97E00E9452116C2F8BEF97E043
:2023A0000E945211CF910C9415108F929F92AF92BF92CF92DF92EF92FF920F931F93CF9375
:2023C000DF9380E00E94811180E10E94811180E40E948111809124088F3F09F46BC030EB7C
:2023E000F32ED0E0C0E08F2D0E94811182E00E94811180E10E94811110E000E0CE01805FD3
:202400009E4F6C01E0912E08F0912F08808190913408892B8083E0913008F091310880818A
:2024200090913508892B8083E0912E08F0912F089081809134088095892380835601A00E01
:20244000B11E20E1E22EF50181915F0190912908992369F18EBD00000DB407FEFDCF8EB5AC
:20246000EA94E110F0CFE0912E08F0912F08808190913408892B8083005F1F4F003811059F
:2024800009F0C0CFC058DF4FF394C115F4E0DF0709F0A9CFDF91CF911F910F91FF90EF90B8
:2024A000DF90CF90BF90AF909F908F9008950E945104D6CF9090B8008CE08093B80090EBAF
:2024C000F92ED0E0C0E0882483948F2D0E94811182E00E94811180E10E94811110E000E0D7
:2024E000CE01805F9E4F5C01809122088092D7078093F9071092D8071092FA0760E48BEFC4
:2025000097E00E9452116501C00ED11E80E1E82EF60161916F018BEF97E00E945211EA94D8
:20252000E110F6CF0E941510005F1F4F00381105D9F6C058DF4FF394C115F4E0DF0729F6B8
:202540009092B800A7CF90E080E00895DC01AA0FBB1FA751BA4FFC01EE0FFF1FE551FA4FB6
:202560002D913C9140815181240F351FFC01EE0FFF1FE351FA4F80819181820F931F08952E
:20258000CF93C82F61E00E94E80561E08C2FCF910C94BA05CF93C82F60E00E94E80560E0EF
:2025A0008C2FCF910C94BA05E0E1F1E080E094E0DF019C011D9221503040E1F70895FC01BC
:2025C00001900020E9F73197AF01481B590BBC0187E098E00C943B05CF93DF930E94060D26
:2025E000EC018EE595E00E94DF128C0F9D1FDF91CF9108958F929F92AF92BF920F931F9377
:20260000CF93DF93CDB7DEB7A1970FB6F894DEBF0FBECDBF19A2423008F44AE08E010F5D00
:202620001F4F842E912CB12CA12CA50194010E94322BE62FB901CA01EA30F4F4E05DD80127
:20264000EE938D01232B242B252B79F790E080E0109719F0CD010E94DF12A1960FB6F894A5
:20266000DEBF0FBECDBFDF91CF911F910F91BF90AF909F908F900895E95CE1CF0C94DF1245
:202680004F925F926F927F928F929F92AF92BF92CF92DF92EF92FF92CF93DF936B017C01D1
:2026A000D42FAC019B010E94E72D882391F081E695E0DF91CF91FF90EF90DF90CF90BF9015
:2026C000AF909F908F907F906F905F904F900C94DF1226013701E89477F82FEF3FEF4FE734
:2026E0005FE7C301B2010E94E72D81110DC02FEF3FEF4FE75FE7C301B2010E94D02B1816FE
:202700001CF485E695E0D5CF2FEF3FEF4FE75FE4C701B6010E942F2D18161CF489E695E0C1
:20272000C8CF2FEF3FEF4FE75FECC701B6010E94D02B87FDF3CF20E030E0A901C701B6019A
:202740000E94D02B912C812C87FF08C08DE20E94210D4C01F7FAF094F7F8F094CD2FA12CE7
:2027600060E070E080E09FE3AD1640F420E030E040E251E40E94D52BA394F6CFA7019601AC
:202780000E94642B2B013C010E944E2C5B016C014AE00E94FA127C01E80CF91CDD23B1F1BA
:2027A000C601B5010E947D2C9B01AC01C301B2010E94632B4B015C018EE20E94210DE80E82
:2027C000F91EC15018F120E030E040E251E4C501B4010E94342D2B013C010E944E2C4B0112
:2027E000B12CA12C4AE0C501B4010E94FA12E80EF91EC501B4010E947D2C9B01AC01C301FC
:20280000B2010E94632B4B015C01DBCFC701DF91CF91FF90EF90DF90CF90BF90AF909F9051
:202820008F907F906F905F904F9008950E943E2E85ED8093BC008091D3079091D407A09199
:20284000D507B091D6070796A11DB11D23E0B695A795979587952A95D1F72091BC0024FD6E
:2028600003C01092D10708954091D3075091D4076091D5077091D607452B462B472B69F3BD
:202880000097A105B10541F025E32A95F1F700000197A109B109E1CF8091D2070C94F40F2C
:2028A0000C94BB2A80916E0590916F05181619060CF04CC080916E0590916F052091E8056E
:2028C0003091E905821B930B90936F0580936E0580916E0590916F0597FF38C06091A407AE
:2028E0007091A50790E080E00E945014609181077091820781E090E00E94501460919C07E7
:2029000070919D0782E090E00E9450146091A6077091A70783E090E00E9450146091A1077B
:2029200084E090E00E9450146091A00785E090E00E94501460919F0786E090E00E945014D7
:2029400060919E0787E090E00C94501408950C94B32A2F923F924F925F926F927F928F9255
:202960009F92AF92BF92CF92DF92EF92FF920F931F93CF93DF93CDB7DEB763970FB6F89424
:20298000DEBF0FBECDBFEBEECE2EE5E0DE2E2BE737E076010FEF13E01A82198240E050E083
:2029A000BA01F701819191917F014C01092E000CAA08BB08480D591D6A1D7B1D8017910792
:2029C0000CF48C01E981FA81E817F90714F49A8389832E153F0529F729813A813093E7059A
:2029E0002093E6051093E5050093E405CB01BA01665F7F4F8F4F9F4F24E130E040E050E0E5
:202A00000E94C92A3093A3072093A207C901059666EF7FEF0E94012EAB01812C912C5401F4
:202A2000F601A191B1916F01A40FB51F9D010E941B2E860E971EA81EB91EEE16FF0681F744
:202A4000C501B40128EC30E040E050E00E94C92ACA01B9010E947F2C0E94A72D0E94472C95
:202A6000709391076093900781E390E090937C0780937B0789819A81800F911FAC0197FD7D
:202A8000019695958795EBE4F6E021E330E02639310509F429C1A0919C07B0919D07619179
:202AA0007191AB2B09F014C1681779070CF019C160817181681779070CF413C130937C07AF
:202AC00020937B0781E080938B0729813A81201B310B2630310514F410928B07CA01880FB5
:202AE000991F480F591F57FF02C04F5F5F4FCA01959587959B8B8A8B812C912C54011F822F
:202B00001E82750164011D821C821E861F86188A198A1B827724739422242394312CC10114
:202B20000E94A6128C01F1013196F987E887772009F4ECC02A893B89281739070CF443C1CC
:202B4000CF010E94A6129A838983EA89FB89E817F9070CF038C1E01BF10B8F01BF01FF0FE2
:202B6000880B990B0E947F2C2B013C0169817A812A893B89621B730B600F711F072E000CD1
:202B8000880B990B0E947F2C9B01AC01C301B2010E94D52B2B013C01B101330C880B990BBE
:202BA0000E947F2C9B01AC01C301B2010E94642B6A877B878C879D873B81332309F49DC041
:202BC0002E853F85488959890E94632B4B015C018C819D8101969D838C83712C31E03B8395
:202BE0002884398426EC2216310409F098CFEC81FD81BF01FF0F880B990B0E947F2C9B01B4
:202C0000AC01C501B4010E94D52B4B015C01E0918107F0918207EE0FFF1FEE0FFF1FE85FC1
:202C2000FD4F2591359145915491C501B4010E94342D20E030E048EC51E40E94D52B9B01DC
:202C4000AC0160E070E080E89FE30E94D52B60938707709388078093890790938A072E8192
:202C60003F81B901330F880B990B0E947F2C9B01AC01C701B6010E94D52B20E030E048EC66
:202C800052E40E94342DA50194010E94D52B609383077093840780938507909386076396CB
:202CA0000FB6F894DEBF0FBECDBFDF91CF911F910F91FF90EF90DF90CF90BF90AF909F9014
:202CC0008F907F906F905F904F903F902F9008958617970734F460817181861797070CF061
:202CE000EDCE2F5F3F4FD3CE84E690E090937C0780937B0710928B07E8CE9A859E87EB85A9
:202D0000EF87FC85F88B2D85298B67CF8A899B89081719070CF464CF888599850E94A6126F
:202D20009A838983EA89FB898E179F070CF058CFFB81FF2309F447C02A893B89021B130BB1
:202D4000B801012E000C880B990B0E947F2C2B013C016A897B8989819A81681B790B600F00
:202D6000711F072E000C880B990B0E947F2C9B01AC01C301B2010E94D52B2B013C01B10181
:202D8000330C880B990B0E947F2C9B01AC01C301B2010E94642B2A853B854C855D850E94BB
:202DA000632B9B01AC01C701B6010E94642B6B017C01EE81FF813196FF83EE837724739458
:202DC000F1E0FB830DCF772473940ACFCF92DF92EF92FF9287E00E949105892B09F038C025
:202DE00081E090E09093A9078093A807E0918107F0918207EE0FFF1FE051FE4F65917491D6
:202E000085E091E00E947528E091A407F091A507EE0FFF1FE452FE4F659174918BE091E0DF
:202E20000E947528E091A407F091A507EA30F10508F066C0E25EF84E0C94152E7A174E187C
:202E40002D178517C317011853189118CF180D191092A9071092A807C9CF8091A807909162
:202E6000A907892BA9F48EEC93E09093800780937F0788E893E190938F0780938E0710923A
:202E80007E0710927D0710928D0710928C0732C060919E0770919F07072E000C880B990B75
:202EA0000E947F2C6B017C012DE13CE947ED53E40E94642B0E94472C7093800760937F07F5
:202EC00084EC99E090938F0780938E072DE13CE947ED53E4C701B6010E94632B0E94472C46
:202EE00070937E0760937D078CE396EF90938D0780938C0781E090E090939B0780939A0738
:202F0000FF90EF90DF90CF9008958091A8079091A907892B49F485E891E09093800780931B
:202F20007F0780ED97E0A7CF60919E0770919F07072E000C880B990B0E947F2C6B017C01C6
:202F400024EE3CE74CE253E40E94642B0E94472C7093800760937F0788EE93E090938F07EC
:202F600080938E0724EE3CE74CE253E4C701B6010E94632B0E94472C70937E0760937D074C
:202F800088E19CEFB3CF8091A8079091A907892B49F482EC90E09093800780937F0788EEA2
:202FA00093E069CF60919E0770919F07072E000C880B990B0E947F2C6B017C0124EE3CE746
:202FC0004CEA52E40E94642B0E94472C7093800760937F0784EF91E090938F0780938E07F7
:202FE00024EE3CE74CEA52E4C701B6010E94632B0E94472C70937E0760937D078CE09EEF74
:2030000075CF8091A8079091A907892BA9F486E793E09093800780937F0784EF91E0909360
:203020008F0780938E0710927E0710927D0710928D0710928C0732C06091A0077091A10767
:20304000072E000C880B990B0E947F2C6B017C012AE23BE246EC53E40E94642B0E94472CEA
:203060007093800760937F078AEF90E090938F0780938E072AE23BE246EC53E4C701B601F2
:203080000E94632B0E94472C70937E0760937D0786E09FEF90938D0780938C0710929B0757
:2030A00010929A072DCF8091A8079091A907892B49F482E691E09093800780937F0788ECBF
:2030C00090E0ADCF6091A0077091A107072E000C880B990B0E947F2C6B017C012FEE38E8D8
:2030E0004EE153E40E94642B0E94472C7093800760937F0784E690E090938F0780938E07E6
:203100002FEE38E84EE153E4C701B6010E94632B0E94472C70937E0760937D078CE99FEF46
:20312000B9CF8091A8079091A907892B49F481EB90E09093800780937F0784E690E06FCF4E
:203140006091A0077091A107072E000C880B990B0E947F2C6B017C012FEE38E84EE952E4D6
:203160000E94642B0E94472C7093800760937F0782E390E090938F0780938E072FEE38E893
:203180004EE952E4C701B6010E94632B0E94472C70937E0760937D078EEC9FEF7BCF80919C
:2031A000A8079091A907892B49F488E590E09093800780937F0782E390E031CF6091A00711
:2031C0007091A107072E000C880B990B0E947F2C6B017C012FEE38E84EE152E40E94642BC5
:2031E0000E94472C7093800760937F0789E190E090938F0780938E072FEE38E84EE152E4DA
:20320000C701B6010E94632B0E94472C70937E0760937D0787EE9FEF3DCF8091A8079091FB
:20322000A907892B49F483E290E09093800780937F0784E190E0F3CE6091A0077091A107FE
:20324000072E000C880B990B0E947F2C6B017C0124EE37EA4DE751E40E94642B0E94472CDE
:203260007093800760937F078AE090E090938F0780938E0724EE37EA4DE751E4C701B601F5
:203280000E94632B0E94472C70937E0760937D0786EF9FEFFFCE1F920F920FB60F9211242D
:2032A0002F933F938F939F93AF93BF938091D5059091D605A091D705B091D8053091D405E6
:2032C00023E0230F2D3758F50196A11DB11D2093D4058093D5059093D605A093D705B0931C
:2032E000D8058091D9059091DA05A091DB05B091DC050196A11DB11D8093D9059093DA05B9
:20330000A093DB05B093DC05BF91AF919F918F913F912F910F900FBE0F901F90189526E891
:20332000230F0296A11DB11DD2CF1F920F920FB60F9211242F933F934F935F936F937F932D
:203340008F939F93AF93BF93EF93FF93E0910301F09104010995FF91EF91BF91AF919F9108
:203360008F917F916F915F914F913F912F910F900FBE0F901F9018951F920F920FB60F929E
:2033800011242F933F934F935F936F937F938F939F93AF93BF93EF93FF93E0910101F0918C
:2033A00002010995FF91EF91BF91AF919F918F917F916F915F914F913F912F910F900FBEA0
:2033C0000F901F9018951F920F920FB60F9211242F933F934F935F936F937F938F939F9335
:2033E000AF93BF93EF93FF938091B900887F803609F44AC0F0F5883209F4A7C018F58031D6
:2034000009F49BC0B8F4882309F4F9C0883009F494C0FF91EF91BF91AF919F918F917F913E
:203420006F915F914F913F912F910F900FBE0F901F901895883109F488C0803251F78093BA
:20344000CF0714C0803409F49DC040F48033B9F38833F9F68093CF0785ECB0C0803509F4FB
:2034600085C0883509F496C0883499F60E941814D0CF883909F48CC038F5883729F050F4EC
:20348000883611F0803729F683E08093D1071092D30557C0883809F47BC0803919F0803846
:2034A00009F0B7CF8091D305803208F071C0E091D30581E08E0F8093D3058091BB00F0E0FB
:2034C000ED54FA4F80833DC0803B39F0E0F4803A09F479C0883A09F09CCF84E08093D10745
:2034E0001092B2051092B105E091DF05F091E00509958091B10581110FC081E08093B10570
:203500001092910509C0803C09F4A6CF883C09F4A3CF883B09F07DCFE091B20581E08E0F1B
:203520008093B205F0E0EF56FA4F80818093BB009091B2058091B10529C08091AC07809335
:20354000BB0085EC8093BC0064CF9091CE078091CD07981758F5E091CE0781E08E0F80930F
:20356000CE07F0E0E355F84F8081E9CFE091CE0781E08E0F8093CE078091BB00F0E0E3556E
:20358000F84F80839091CE078091CD079817C8F285E8D8CFE091CE0781E08E0F8093CE075D
:2035A0008091BB00F0E0E355F84F80838091D00781115CCF81E08093AB0784EA8093BC00E5
:2035C0001092D10726CF85EC8093BC001092D1078091D305803230F4E091D305F0E0ED54A9
:2035E000FA4F10826091D30570E0E091DD05F091DE0583EB95E009951092D3050ACF1092AA
:20360000CF0734CFEBEFF7E01382128288EE93E0A0E0B0E084839583A683B78384E295E0A1
:2036200091838083E7E0F8E01382128220E830E03583248380E490E09783868331872087DE
:2036400093878287168A158614861786168681E0858B848B2FEF3FEF338B228B318B208B9B
:20366000878B108E128E118E86E395E0918380838FEF858F81A3878F868F80A30895CF9363
:20368000DF9300D000D0CDB7DEB7789484B5826084BD84B5816084BD85B5826085BD85B5A4
:2036A000816085BD80916E00816080936E0010928100809181008260809381008091810049
:2036C000816080938100809180008160809380008091B10084608093B1008091B000816064
:2036E0008093B00080917A00846080937A0080917A00826080937A0080917A008160809392
:203700007A0080917A00806880937A001092C10062E082E00E94E80562E087E00E94E80561
:2037200062E088E00E94E80562E089E00E94E80562E08AE00E94E80562E08BE00E94E8059F
:2037400061E08DE00E94E80560E08CE00E94E80560E080E10E94E80560E081E10E94E80590
:203760008BB187788BB98AB188678AB985B185B984B184B988B188B987B187B982E0809310
:2037800023088CE380932208809124088F3F09F4B0C161E0809126080E94E80561E0809178
:2037A00028080E94E80580912808082E000C990BFC01E258F84FE491F0E0EE0FFF1FEC5801
:2037C000F84F2591349130932F0820932E08FC01E05AF84FE491E093340880912608082E2D
:2037E000000C990BFC01E258F84FE491F0E0EE0FFF1FEC58F84F2591349130933108209386
:203800003008FC01E05AF84FE491E09335088091290881113EC061E0809124080E94E805EE
:2038200061E0809125080E94E80580912508082E000C990BFC01E258F84FE491F0E0EE0F96
:20384000FF1FEC58F84F2591349130932D0820932C08FC01E05AF84FE491E09333088091B3
:203860002408082E000C990BFC01E258F84FE491F0E0EE0FFF1FEC58F84F2591349130938F
:203880002B0820932A08FC01E05AF84FE491E093320880912908882309F43BC02FB72983F9
:2038A000F8948091E305811127C0E8E8F7E08491EAE6F7E09491E82FF0E0EE0FFF1FEA5A3C
:2038C000F84FA591B491EC91E92321F461E08AE00E94BA0561E08AE00E94E8058CB5806120
:2038E0008CBD8CB580648CBD61E08DE00E94E80561E08BE00E94E8058091E3058F5F80939F
:20390000E30539813FBF8CB58C7F8CBD8DB581608DBD61E0809127080E94E80561E08091A3
:2039200027080E94BA0561E070E080E090E00E94680660E0809127080E94BA056AE070E00B
:2039400080E090E00E94680661E0809127080E94BA058EEA0E94811185ED0E94811180E8EB
:203960000E94811188EA0E9481118FE30E94811183ED0E94811180E00E94811180E40E9489
:2039800081118DE80E94811184E10E94811180E20E94811180E00E94811181EA0E9481118A
:2039A00088EC0E9481118AED0E94811182E10E94811181E80E9481118FEC0E94811189ED5B
:2039C0000E94811181EF0E9481118BED0E94811180E40E94811184EA0E94811186EA0E9417
:2039E00081118FEA0E94811188E00E949105892B09F096C081E080930001EE24E394F12CCA
:203A000084E1A82EB12C90E1C92ED12C23E2822E912C3EE1232E312C84E690E09A838983E7
:203A2000412C512C320181E00E942C06092E000CAA0BBB0B480E591E6A1E7B1EE981FA81A3
:203A40003197FA83E983EF2B71F70E94D412F0921A08E0921908F0921808E0921708B092FF
:203A60001408A0921308D0921608C092150881E080931B0880931C0884E997E00E94EC129C
:203A800090921408809213083092160820921508F2E0F0931B08F0931C08C301B2010E94D4
:203AA0007F2C20E030E048EC52E40E94D52B20E030E040EA50E40E94342D20E030EC4FE77C
:203AC00054E40E94D52B02E917E022E044E00E945728C8010E943E1382E997E00E94EC12A5
:203AE0000E94D51166E970E080E090E00E94680693CF1092E2051092E1051092D807109229
:203B0000FA070E94D60F89E395E09093E0058093DF058AE395E09093DE058093DD05F9CE99
:203B200089E00E949105892B09F005C183E080930001EE24E394F12CB2E03B2E16E1C12E73
:203B4000D12C61E08DE00E94BA050E94D412F0921A08E0921908F0921808E09217081092C5
:203B6000140810921308109216081092150881E080931B0880931C0887E00E9491050197E8
:203B800009F048C080E190E00E94CA1281E190E00E94CA128CE090E00E94CA1280E00E9429
:203BA0002C068C018FEB97E00E94EC1224E130E03093140820931308D0921608C092150804
:203BC00030921B0830921C08B801110F880B990B0E947F2C20ED3CEC48EB5BE30E94342D14
:203BE00002E917E022E044E00E945728C8010E943E138DEB97E00E94060D0E94D51160E074
:203C00008DE00E94BA0566E970E080E090E00E94680697CF80E190E00E94C01281E190E0DA
:203C20000E94CA128CE090E00E94CA1280917A00887F80937A0080917A00876080937A008E
:203C40000BEE15E080E00E942C06F801819391938F0187E591E00197F1F72BE737E02E17B6
:203C60003F0781F70E94A9146091900770919107072E000C880B990B0E947F2C23E531EB1D
:203C80004EEC5BE30E94342D2B013C016091E6057091E7058091E4059091E505681B790B6B
:203CA000072E000C880B990B0E947F2C23E531EB4EEC5BE30E94342D4B015C018DEA97E009
:203CC0000E94EC1230921B0830921C0802E917E022E044E0C301B2010E94572884E190E004
:203CE000909314088093130880E190E09093160880931508C8010E943E1388EA97E00E94CE
:203D0000EC1222E044E0C501B4010E945728E4E1F0E0F0931408E093130826E230E0309346
:203D2000160820931508C8010E943E1384EA97E00E94EC1262CF8AE00E949105892B09F0D4
:203D400001C183E080930001EE24E394F12CE2E03E2EF6E1CF2ED12C61E08DE00E94BA0576
:203D60000E94D412F0921A08E0921908F0921808E092170810921408109213081092160816
:203D80001092150881E080931B0880931C0887E00E949105019709F046C080E190E00E94ED
:203DA000CA1281E190E00E94CA120E94240680E00E942C068C018BEE97E00E94EC1284E155
:203DC00090E09093140880931308D0921608C092150830921B0830921C08B801110F880BE0
:203DE000990B0E947F2C2DE839E142E55DE30E94342D02E917E021E044E00E945728C80148
:203E00000E943E1389EE97E00E94060D0E94D51160E08DE00E94BA0566E970E080E090E007
:203E20000E94680699CF80E190E00E94CA1281E190E00E94C0120E94240680917A00887F17
:203E400080937A0080917A00876080937A000BEE15E080E00E942C06F801819391938F01F3
:203E600087E591E00197F1F72BE737E02E173F0781F70E94A9146091900770919107072E04
:203E8000000C880B990B0E947F2C2CE437E74DE65DE30E94342D2B013C016091E6057091A8
:203EA000E7058091E4059091E505681B790B072E000C880B990B0E947F2C2CE437E74DE6E4
:203EC0005DE30E94342D4B015C0188ED97E00E94EC1230921B0830921C0802E917E021E0BC
:203EE00044E0C301B2010E94572884E190E0909314088093130880E190E09093160880939F
:203F00001508C8010E943E1383ED97E00E94EC1221E044E0C501B4010E945728E4E1F0E0EB
:203F2000F0931408E093130826E230E03093160820931508C8010E943E138FEC97E00E943B
:203F4000EC1264CF90E080E00E94A7148A3008F083E090E09093A5078093A40781E090E020
:203F60000E94A7148C3008F083E090E0909382078093810782E090E00E94A714811181E0F4
:203F800090E090939D0780939C0783E090E00E94A714833008F081E090E09093A7078093A4
:203FA000A60784E090E00E94A714E82FF0E03E2F22273A83298385E090E00E94A714E98181
:203FC000FA81E82BFA83E9839F012E5531402D32314020F022E532E03A83298389819A814F
:203FE0009093A1078093A00786E090E00E94A714E82FF0E03E2F22273A83298387E090E02C
:204000000E94A714E981FA81E82BFA83E9839F012E5531402D32314020F022E232E03A831B
:20402000298389819A8190939F0780939E0783E0809300018CE794E0909302018093010195
:20404000809169008C7F826080936900E89A0E94D41281E090E090931A0880931908909306
:204060001808809317088AE090E0909314088093130810921608109215088FE098E00E949F
:20408000EC1288E090E0909314088093130884E190E090931608809315088CEF97E00E9403
:2040A000EC120E94D51168EB7BE080E090E00E9468060E94D41281E080931B0880931C0896
:2040C0008091A8079091A907181619060CF03FC080919A0790919B07019749F481E190E0EB
:2040E0000E94C01280E190E00E94CA1208C081E190E00E94CA1280E190E00E94C0120E94FE
:20410000E61661E08DE00E94BA0580919A0790919B07019719F50E9424061092EA05E091AB
:204120008107F0918207EC30F10508F045C0E556FF4D0C94152EB3206B249224B924E0247B
:2041400007252E2555257C25AB25AB25AB2580E190E00E94CA1281E190E0C6CF8CE090E0C3
:204160000E94CA12DACF8CE796E09093E9058093E80580917A00887F80937A0080917A0074
:20418000876080937A000BEE15E080E00E942C06F801819391938F018BE39BE70197F1F758
:2041A0008091EA05882319F01092EA0505C02BE737E02E173F0749F760E08DE00E94BA05F3
:2041C0000E94E6160E94A9140E94D41281E090E090931A088093190890931808809317089B
:2041E00001E010E027E330E049E050E06AE170E087E098E00E949B0623E030E049E050E052
:204200006FE770E087E098E00E949B0623E030E04DE350E06FE770E087E098E00E949B069B
:2042200027E030E049E050E068E170E087E098E00E94F80722E030E044E250E068E170E0F4
:2042400087E098E00E94F80727E030E04FE350E068E170E087E098E00E94F80723E030E039
:2042600049E050E063E370E087E098E00E94F80723E030E04FE350E063E370E087E098E0E5
:204280000E94F80723E030E049E050E06CE470E087E098E00E94F80723E030E04FE350E07C
:2042A0006CE470E087E098E00E94F80723E030E049E050E065E670E087E098E00E94F80757
:2042C00023E030E04FE350E065E670E087E098E00E94F80725E030E049E050E06BE770E03E
:2042E00087E098E00E94F80725E030E04FE350E06BE770E087E098E00E94F807EAE1F0E00A
:20430000FA83E98301E010E022E030E044E250E069817A8187E098E00E94F80729813A81B1
:204320002B5F3F4F3A8329832338310559F786E690E09A8389834AE0E42EF12C01E010E0EC
:2043400022E030E0A70169817A8187E098E00E949B0695E0E90EF11CE1E4EE16F10471F7FD
:2043600029813A81295131093A8329832B31310511F780918107909182070A970CF022C45B
:204380001A821982E0907D07F0907E070F2C000C000B110B20907B0730907C0789819A81E5
:2043A000280E391E40907F0750908007052C000C660877084E185F08600A710AF101EE0FE8
:2043C000FF1FE757FA4F20813181032E000C440B550B2E193F09400B510BAAECBFEF0E94DD
:2043E000F62AA30192010E94C92A49015A019FE3890E911CA11CB11CE0E48E169104A1043A
:20440000B1042CF02FE3822E912CA12CB12CF9E08F169104A104B1042CF499E0892E912C28
:20442000A12CB12CC980DA802CE1C20ED11CF101EE0FFF1FE957FA4F20813181032E000C3F
:20444000440B550B2E193F09400B510BAAECBFEF0E94F62AA30192010E94C92ABA01A90140
:20446000415C5F4F6F4F7F4F403451056105710524F04FE350E060E070E049305105610584
:20448000710524F449E050E060E070E089819A814B96EE24E394F12C84019601BC0187E0B9
:2044A00098E00E94850D89819A8101969A8389838336910509F066CF109214081092130873
:2044C00010921608109215088091A8079091A907892B09F0C5C483E498E00E94060D8FE093
:2044E00090E0909314088093130810921608109215088BE091E00E943E138091A6079091B2
:20450000A707892B01F501E010E02BE130E047E050E06DE070E087E098E00E94F80722E0E0
:2045200030E045E050E06DE070E087E098E00E949B0622E030E045E050E067E270E087E0F0
:2045400098E00E949B068AE290E09093140880931308109216081092150885E091E00E9460
:204560003E138091A6079091A707019701F501E010E021E230E047E050E068E270E087E093
:2045800098E00E94F80722E030E045E050E068E270E087E098E00E949B0622E030E045E0A8
:2045A00050E068E470E087E098E00E949B068BE490E090931408809313081092160810925F
:2045C000150880919C0790919D07892B09F04BC488E10E94210D8091A6079091A70702972A
:2045E00001F501E010E02BE030E047E050E068E470E087E098E00E94F80722E030E045E02F
:2046000050E068E470E087E098E00E949B0622E030E045E050E062E570E087E098E00E942D
:204620009B068091A8079091A907892B09F028C486E590E0909314088093130810921608A7
:20464000109215088DE398E00E94060D80919A0790919B076091A2077091A307019709F0B3
:2046600004C4072E000C880B990B0E947F2C2DE839E142E55DE30E94342D20E030E040E2E2
:2046800051E40E94D52B6B017C0120E030E040E251E40E94D02B02E917E022E087FF21E0EB
:2046A00044E0C701B6010E94572882E690E09093140880931308109216081092150882E907
:2046C00097E00E943E1388E398E00E94060D60918E0770918F07072E000C880B990B0E94A1
:2046E0007F2C20E030E048EC52E40E94D52B2091A4073091A507243031050CF0F1C302E905
:2047000017E020E044E00E945728109214081092130889E090E0909316088093150882E92D
:2047200097E00E943E1360918E0770918F0780918C0790918D07680F791F072E000C880BB6
:20474000990B0E947F2C20E030E048E453E40E94D52B2091A4073091A507243031050CF004
:20476000CCC302E917E020E044E00E945728109214081092130881E290E0909316088093E1
:20478000150882E997E00E943E1360918C0770918D07072E000C880B990B0E947F2C20E049
:2047A00030E048EC52E40E94D52B2091A4073091A507243031050CF0ADC302E917E020E03C
:2047C00044E00E945728109214081092130889E390E0909316088093150882E997E00E9448
:2047E0003E1380918B07F12CE12C8111BBC308E010E028E130E04EE050E06CE570E087E034
:2048000098E00E941A0E8CE590E090931408809313088EE090E0909316088093150881E355
:2048200098E00E94060D0E94D5110E9452148091AA07882309F431C4F12CE12C08E010E05A
:2048400028E130E04BE050E06AE270E087E098E00E941A0E8AE290E0909314088093130856
:204860008BE090E0909316088093150886E498E00E94060D0E94D5118091A8079091A9073C
:2048800018161906A4F688E00E949105892BE1F42091A4073091A5078091A2079091A307BA
:2048A0006AE070E00E94012E253031050CF4F0C37093A1076093A0070E9452141092A707B2
:2048C0001092A6071092AA076AE070E080E090E00E946806ACCF8CE593E09093E905809339
:2048E000E80580917A00887F80937A0080917A00876080937A000BEE15E080E00E942C068B
:20490000F801819391938F018BE49CE30197F1F78091EA05811148CC2BE737E02E173F070E
:2049200061F74ACC8CEC91E09093E9058093E80580917A00887F80937A0080917A0087607E
:2049400080937A000BEE15E080E00E942C06F801819391938F018BE59DE10197F1F7809168
:20496000EA05811129CC2BE737E02E173F0761F723CC8CED90E09093E9058093E8058091BB
:204980007A00887F80937A0080917A00876080937A000BEE15E080E00E942C06F8018193DB
:2049A00091938F0183EB9AE00197F1F78091EA05811102CC2BE737E02E173F0761F7FCCBA8
:2049C0008CE890E09093E9058093E80580917A00887F80937A0080917A00876080937A00C4
:2049E0000BEE15E080E00E942C06F801819391938F0187E794E00197F1F78091EA058111E0
:204A0000DBCB2BE737E02E173F0761F7D5CB84E690E09093E9058093E80580917A00887FC7
:204A200080937A0080917A00876080937A000BEE15E080E00E942C06F801819391938F0107
:204A400087E591E00197F1F78091EA058111B4CB2BE737E02E173F0761F7AECB8CE490E083
:204A60009093E9058093E80580917A00887F80937A0080917A00866080937A00EBEEF5E05A
:204A8000FA83E98380E00E942C06E981FA8181939193FA83E98387E590E00197F1F72BE785
:204AA00037E02E173F0771F787CB84E490E09093E9058093E80580917A00887F80937A0092
:204AC00080917A00856080937A00EBEEF5E0FA83E98380E00E942C06E981FA8181939193F1
:204AE000FA83E98383E290E00197F1F72BE737E02E173F0771F760CB80E490E09093E9054C
:204B00008093E80580917A00887F80937A0080917A00846080937A00EBEEF5E0FA83E983E3
:204B200080E00E942C06E981FA8181939193FA83E9838BE090E00197F1F7000000000000E0
:204B4000000000000000000000002BE737E02E173F0731F731CB8EE390E09093E905809378
:204B6000E80580917A00887F80937A0080917A00826080937A00EBEEF5E0FA83E98380E038
:204B80000E942C06E981FA8181939193FA83E983000000000000000000000000000000003B
:204BA0000000000000000000000000000000000000000000000000002BE737E02E173F0741
:204BC000F1F6FACA80918107909182070A9709F0A0C01BE1C12ED12C312C212CE0907D0767
:204BE000F0907E070F2C000C000B110BE0917B07F0917C07E20DF31DFC83EB8340907F0709
:204C000050908007052C000C660877084E185F08600A710A96012E5F3F4F3A832983EE0F39
:204C2000FF1FE554FA4F20813181032E000C440B550B2E193F09400B510BAAECBFEF0E9479
:204C4000F62AA30192010E94C92A49015A018FE3880E911CA11CB11C90E489169104A10437
:204C6000B1042CF0AFE38A2E912CA12CB12CE9E08E169104A104B1042CF4F9E08F2E912CE3
:204C8000A12CB12C2B813C81220F331F27543A4FF90120813181032E000C440B550B2E19FA
:204CA0003F09400B510BAAECBFEF0E94F62AA30192010E94C92ABA01A901415C5F4F6F4FC5
:204CC0007F4F403451056105710524F04FE350E060E070E0493051056105710524F449E06E
:204CE00050E060E070E0EE24E394F12C840129813A81B60187E098E00E94850DFFEF2F1A63
:204D00003F0AC980DA8022E32216310409F066CFD3CB80918107909182070B9709F0CCCBF4
:204D20006BE1C62ED12C312C212CE0907D07F0907E070F2C000C000B110B80917B07909171
:204D40007C07820D931D9C838B8340907F0750908007052C000C660877084E185F08600A46
:204D6000710AF6013496FA83E983FC01EE0FFF1FED52FA4F20813181032E000C440B550B2F
:204D80002E193F09400B510BAAECBFEF0E94F62AA30192010E94C92A49015A01FFE38F0EE7
:204DA000911CA11CB11C20E482169104A104B1042CF04FE3842E912CA12CB12C39E0831618
:204DC0009104A104B1042CF439E0832E912CA12CB12C8B819C81880F991F8F529A4FFC0154
:204DE00020813181032E000C440B550B2E193F09400B510BAAECBFEF0E94F62AA301920101
:204E00000E94C92ABA01A901415C5F4F6F4F7F4F403451056105710524F04FE350E060E065
:204E200070E0493051056105710524F449E050E060E070E0EE24E394F12C840129813A81E6
:204E4000B60187E098E00E94850DFFEF2F1A3F0AC980DA8029E12216310409F066CF2CCBC9
:204E600080E498E03ACB89E1B4CB072E000C880B990B0E947F2C20ED3CEC48EB5BE3FBCB37
:204E800086E590E0909314088093130810921608109215088AE398E00E94060D80919A07FF
:204EA00090919B076091900770919107019769F4072E000C880B990B0E947F2C2CE437E726
:204EC0004DE65DE30E94342DDECB072E000C880B990B0E947F2C23E531EB4EEC5BE3F2CF91
:204EE0002091A4073091A50702E917E02830310514F421E007CC22E005CC2091A4073091AD
:204F0000A50702E917E02830310514F421E02CCC22E02ACC2091A4073091A50702E917E0D1
:204F20002830310514F421E04BCC22E044E00E9457288091A8079091A907181619060CF0A2
:204F400042CC80919407809393078091950780939407809196078093950780919707809370
:204F6000960731CC09E010E029E130E04CE050E06BE570E087E098E00E941A0E8CE590E01E
:204F800090931408809313088DE090E09093160880931508C0908707D0908807E090890789
:204FA000F0908A072DEC3CEC47EC52E4C701B6010E94D02B87FF33C041E050E0C701B601D1
:204FC0000E9440138EE298E00E94060DF12CE12C0AE010E029E130E045E150E061E670E034
:204FE00087E098E00E941A0E82E690E090931408809313088AE190E0909316088093150877
:205000006091830770918407809185079091860741E050E00E94401383E298E002CC2AE93A
:2050200039EF49E754E4C701B6010E94D02B87FF09C050E040E0C701B6010E9440138BE244
:2050400098E0C2CF20E030E04AE754E4C701B6010E94D52B4B015C012AE93FE34CE156E468
:20506000C701B6010E94D02B87FF09C042E050E0C501B4010E94401388E298E0A5CF41E08C
:2050800050E0C501B4010E94401385E298E09CCF70939F0760939E070FCC80E090E0892B86
:2050A00011F40C9460200E9400000C946020EF920F931F93CF93DF93E80134E047FD34E10A
:2050C000042E000C550B57FF03C0519541955109E32E022F242FAE010E947C28CE01DF913A
:2050E000CF911F910F91EF900895FB01DC0105900D920020E1F70895A9E0B0E0E2E8F8E285
:205100000C94012B6A01F22EB02E102FFBE3AF2EA01608F41BE31F5F012F27E0AE014F5F9E
:205120005F4F0E94DB29BC018981982F9970913009F43FC09BE2E1FC04C09E2D9170E0FC01
:205140003AC05E2D5071E82FE87083FF46C084E0911101C083E0EF2DE81B8F1508F0E0E06D
:20516000D6018E2F20E2552351F1992329F0D6019C93C60101966C0196012D5F3F4FE2FEA8
:2051800024C08EE4D6018C9391E411969C93119712968C93D9018E2F90E281111BC0E20FA2
:2051A000F32FF11D10828EEF9FEF2996ECE00C941D2B9DE2C6CF90E2C4CF2D938150811173
:2051C000FCCFCE0ED11CE0E0D0CF8EE6D6018C9391E6DBCF9D938150E0CF482F447082FFF5
:2051E0003DC084E0911101C083E08F1510F4EF2DE81BD6018E2F20E2552309F1992329F0E4
:20520000D6019C93C60101966C0196012D5F3F4FE2FE1BC089E4D6018C938EE411968C93B6
:20522000119786E412968C93D9018E2F90E2882309F4B5CF9D938150FACF2D938150811173
:20524000FCCFCE0ED11CE0E0D9CF89E6D6018C938EE611968C93119786E6E4CF9B0177FFDA
:2052600002C030E020E0A1E0B0E0911102C0B0E0A0E0F9013196AE0FBF1F8B2C912CBB202C
:2052800009F461C05401EFEFAE1ABE0AAA0DBB1DFA161B0619F014F04F2D4A1B511188C0D5
:2052A000E3FC59C07601A42FB0E2A1114FC0C40ED11C992309F45BC040E0D6011196F60131
:2052C00090836D01552309F448C0012F060F9A81582F507184FF03C0913309F401501016AA
:2052E0000CF047C0093008F008E0EEE2FE2E5B01A01AB10885019194819491082F3F3207C7
:2053000029F4D601FC92F60131966F016217730794F1021713077CF5DB01A21BB30BAA249C
:20532000A394B12CAC0EBD1EAA0DBB1D11968C9121503109D601119628153905F4F0F601F2
:2053400080836D01DBCFB12CA12CA0CFF701B1937F01A150AACF9111B0CFD601942F50E305
:2053600002C05D9391509111FCCFC40ED11C40E0ACCF01E0BACF80E3DBCF6217730731F444
:20538000963388F4953311F4552369F0F6018083FD01842F90E2811108C0A40FB11D1C9284
:2053A00090E080E002CF81E3F1CF91938150F3CF911183CF8ACF283008F027E03327DA0198
:2053C000990F311D87FD916000966105710539F432602E5F3D9330E32A95E1F708959F3FAF
:2053E00030F080387105610509F03C5F3C5F3D93913008F08068911DDF93CF931F930F9383
:20540000FF92EF92192F987F9695E92F96959695E90FFF27EE53FF4F99273327EE24FF2486
:20542000A701E70105900894079428F4360FE71EF81E491F511D660F771F881F991F0694BA
:20544000A1F70590079428F4E70EF81E491F561FC11D770F881F991F661F0694A1F7059071
:20546000079428F4F80E491F561FC71FD11D880F991F661F771F0694A1F70590079420F4DE
:20548000490F561FC71FD81F990F661F771F881F0694A9F784911095177041F0D695C79585
:2054A00057954795F794E7941A95C1F7E8E6F0E068941590159135916591959105907FE2FA
:2054C0007395E118F10A430B560BC90BD009C0F7E10CF11E431F561FC91FD01D7EF4703300
:2054E00011F48A95E6CFE894015030F0080F0AF40027021708F4202F2395022F7A3328F098
:2055000079E37D932A95E9F710C07D932A9589F6069497956795379517951794E118F10A89
:20552000430B560BC90BD00998F023957E9173957A3308F070E37C932013B8F77E917061EF
:205540007D9330F0839571E37D9370E32A95E1F71124EF90FF900F911F91CF91DF91992792
:2055600087FD90950895F999FECF92BD81BDF89A992780B50895262FF999FECF1FBA92BDF9
:2055800081BD20BD0FB6F894FA9AF99A0FBE01960895052E97FB1EF400940E94E02A57FD0C
:2055A00007D00E94322B07FC03D04EF40C94E02A50954095309521953F4F4F4F5F4F0895A7
:2055C00090958095709561957F4F8F4F9F4F08950E94542BA59F900DB49F900DA49F800D9D
:2055E000911D11240895B7FF0C94E82A0E94E82A821B930B08952F923F924F925F926F92D2
:205600007F928F929F92AF92BF92CF92DF92EF92FF920F931F93CF93DF93CDB7DEB7CA1B8B
:20562000DB0B0FB6F894DEBF0FBECDBF09942A88398848885F846E847D848C849B84AA842A
:20564000B984C884DF80EE80FD800C811B81AA81B981CE0FD11D0FB6F894DEBF0FBECDBFD7
:20566000ED010895A1E21A2EAA1BBB1BFD010DC0AA1FBB1FEE1FFF1FA217B307E407F50746
:2056800020F0A21BB30BE40BF50B661F771F881F991F1A9469F760957095809590959B0138
:2056A000AC01BD01CF010895A29FB001B39FC001A39F700D811D1124911DB29F700D811D61
:2056C0001124911D08955058BB27AA270E947B2B0C94F52C0E94E72C38F00E94EE2C20F03D
:2056E00039F49F3F19F426F40C94E42C0EF4E095E7FB0C94DE2CE92F0E94062D58F3BA17BC
:20570000620773078407950720F079F4A6F50C94282D0EF4E0950B2EBA2FA02D0B01B90146
:2057200090010C01CA01A0011124FF27591B99F0593F50F4503E68F11A16F040A22F232FC1
:20574000342F4427585FF3CF469537952795A795F0405395C9F77EF41F16BA0B620B730B34
:20576000840BBAF09150A1F0FF0FBB1F661F771F881FC2F70EC0BA0F621F731F841F48F492
:20578000879577956795B795F7959E3F08F0B0CF9395880F08F09927EE0F97958795089560
:2057A0000E94BA2C08F481E008950E94E92B0C94F52C0E94EE2C58F00E94E72C40F029F4EA
:2057C0005F3F29F00C94DE2C51110C94292D0C94E42C0E94062D68F39923B1F3552391F3D4
:2057E000951B550BBB27AA2762177307840738F09F5F5F4F220F331F441FAA1FA9F335D044
:205800000E2E3AF0E0E832D091505040E695001CCAF72BD0FE2F29D0660F771F881FBB1FE2
:20582000261737074807AB07B0E809F0BB0B802DBF01FF2793585F4F3AF09E3F510578F0A4
:205840000C94DE2C0C94292D5F3FE4F3983ED4F3869577956795B795F7959F5FC9F7880F46
:20586000911D9695879597F90895E1E0660F771F881FBB1F621773078407BA0720F0621BED
:20588000730B840BBA0BEE1F88F7E09508950E944E2C6894B1110C94292D08950E940E2D4E
:2058A00088F09F5798F0B92F9927B751B0F0E1F0660F771F881F991F1AF0BA95C9F714C07A
:2058C000B13091F00E94282DB1E008950C94282D672F782F8827B85F39F0B93FCCF386954E
:2058E00077956795B395D9F73EF490958095709561957F4F8F4F9F4F0895E89409C097FB13
:205900003EF490958095709561957F4F8F4F9F4F9923A9F0F92F96E9BB279395F6958795D9
:2059200077956795B795F111F8CFFAF4BB0F11F460FF1BC06F5F7F4F8F4F9F4F16C088236A
:2059400011F096E911C0772321F09EE8872F762F05C0662371F096E8862F70E060E02AF0DE
:205960009A95660F771F881FDAF7880F9695879597F90895990F0008550FAA0BE0E8FEEFEC
:2059800016161706E807F907C0F012161306E407F50798F0621B730B840B950B39F40A26E8
:2059A00061F0232B242B252B21F408950A2609F4A140A6958FEF811D811D089597F99F67C1
:2059C00080E870E060E008959FEF80EC089500240A941616170618060906089500240A9404
:2059E00012161306140605060895092E0394000C11F4882352F0BB0F40F4BF2B11F460FF8C
:205A000004C06F5F7F4F8F4F9F4F089557FD9058440F551F59F05F3F71F04795880F97FB6D
:205A2000991F61F09F3F79F087950895121613061406551FF2CF4695F1DF08C01616170611
:205A40001806991FF1CF86957105610508940895E894BB2766277727CB0197F908950E945C
:205A6000BA2C08F48FEF08950E94472D0C94F52C0E94E72C38F00E94EE2C20F0952311F0F0
:205A80000C94DE2C0C94E42C11240C94292D0E94062D70F3959FC1F3950F50E0551F629F18
:205AA000F001729FBB27F00DB11D639FAA27F00DB11DAA1F649F6627B00DA11D661F829F1F
:205AC0002227B00DA11D621F739FB00DA11D621F839FA00D611D221F749F3327A00D611D4D
:205AE000231F849F600D211D822F762F6A2F11249F5750409AF0F1F088234AF0EE0FFF1F81
:205B0000BB1F661F771F881F91505040A9F79E3F510580F00C94DE2C0C94292D5F3FE4F320
:205B2000983ED4F3869577956795B795F795E7959F5FC1F7FE2B880F911D9695879597F956
:205B4000089519F416F40C94E42C0C94EC2D0E940E2DB8F39923C9F3B6F39F57550B87FFA3
:205B60000E94FA2D0024A0E640EA900180585695979528F4805C660F771F881F20F0261711
:205B80003707480730F4621B730B840B202931294A2BA69517940794202531254A2758F7D6
:205BA000660F771F881F20F026173707480730F4620B730B840B200D311D411DA09581F735
:205BC000B901842F9158880F9695879508950E94BA2C880B990B08959F3F31F0915020F4A4
:205BE000879577956795B795880F911D9695879597F9089591505040660F771F881FD2F790
:205C0000089597FB072E16F4009407D077FD09D00E942A2E07FC05D03EF4909581959F4F31
:205C20000895709561957F4F0895EE0FFF1F0590F491E02D09940E94542B332312F48A1B60
:205C40009B0B0C94252E0E94542BB7FF0895821B930B0895AA1BBB1B51E107C0AA1FBB1F28
:205C6000A617B70710F0A61BB70B881F991F5A95A9F780959095BC01CD01089581E090E005
:205C8000F8940C94432EF894FFCF019A069A067878784173007878787800000000000000D0
:205CA0000000000000000000000000000000000000000000000000000000000000000000E4
:205CC000000000000000000000000000000000000000000000000000008080800000000044
:205CE00000000000000000000000008080C0C0000000000000000000000000000000000024
:205D0000000000000000000000000000000000000000000000000000000000000000000083
:205D2000000000000000000000000000000080C0E0F0F8FCF8E00000000000000000000087
:205D400000000000000000808080808000808000000000808080808000FFFFFF0000000046
:205D60008080808000008080000080FFFF8080008080008080808000808000000000008025
:205D80008000008C8E84000080F8F8F88000000000000000000000000000F0F0F0F0F0F05D
:205DA000F0F0F0F0F0F0E0E0C08000E0FCFEFFFFFF7FFFFFFFFFFF000000000000000000F2
:205DC0000000000000FEFFC70101010183FFFF00007CFEC70101010183FFFFFF0038FEC7B8
:205DE0008301010183C7FFFF000001FFFF010100FFFF0701010100007FFF80000000FFFFD0
:205E00007F0000FFFFFF000001FFFFFF0100000000000000000000000000030F3F7F7FFFB9
:205E2000FFFFFFFFFFFFE7C7C78F8F9FBFFFFFC3C0F0FFFFFFFFFFFCFCFCFCFCFCFCFCF833
:205E4000F8F0F0E0C00001030303030301030300000000010303030301010301000000019F
:205E60000303030301010303000000030300000003030000000000000001030303030301F1
:205E8000000000010301000000030301000000000000000000000000000000000080C0E0D6
:205EA000F0F9FFFFFFFFFF3F1F0F87C7F7FFFF1F1F3DFCF8F8F8F87C7DFFFFFFFFFFFFFF05
:205EC000FF7F3F0F0700303000000000000000000000000000000000000000000000FEFE93
:205EE000FC00000000000000000000000000000000000000000000E0C00000000000000006
:205F0000000000003030000000000000000000000000000000000000000000C0FEFFFFFF66
:205F2000FFFFFFFFFFFF7F7F3F1F0F071F7FFFFFF8F8FFFFFFFFFFFEF8E000000001000097
:205F4000000000000000FEFE000000FCFEFC0C06060EFCF80000F0F81C0E0606060CFFFF07
:205F6000FF0000FEFE00000000FCFEFC00183C7E66E6CE84000006FFFF0606FCFEFC0C06A8
:205F800006060000FEFE0000C0F8FC4E4646464E7C7840183C76E6CECC80000000000000D9
:205FA000000000000000000000000000000001070F1F1F3F3F3F3F1F0F030000000000005F
:205FC0000000000000000F0F0000000F0F0F000000000F0F000003070E0C18180C060F0FD4
:205FE0000F0000010F0E0C180C0F070100040E0C180C0F070000000F0F00000F0F0F00008A
:20600000000000000F0F00000007070C0C181C0C060600040E0C180C0F0700000000000098
:20602000000000000000000000000000000000000000000000000000000000000000000060
:20604000000000000000000000000000000000000000000000000000000000000000000040
:20606000000000000000000000000000000000000000000000000000000000000000000020
:206080000000000000000000000000000000000000000000000000000000000103070F1FC7
:2060A0003F7F0080C0E0F0F8FCFE0000000052112511A312D10E1E110B11FC10000000009C
:2060C000340C3B05A312AE0F5509D10EFA0ED20EEE0EE20E010FD10EFA09F9099B06F80729
:2060E0001A0EFD0D850D260D0D0A006E616E00696E66006F76660000FFFFFFFFFFFFFFFFD5
:2061000097E00E94B50DEC81FD81A182FFEF2F1A3F0A2C813D812F5F3F4F3D832C83192DDA
:206120006501320136E92316310409F08FCF07CB1091BE05C090BA05D090BB050D2C000C38
:20614000EE08FF08E091B805F091B905EE0FFF1FEC55FF4F20813181032E000C440B550BEC
:206160002C193D094E095F09A1E1BFEF0E948E362091BC053091BD05032E000C440B550B5E
:206180002C193D094E095F090E94613669017A016FEEC60ED11CE11CF11C80EFC816D1044D
:2061A0001CF07FEEC72ED12CD7FE02C0D12CC12CC092BE055EEB652E55E0752E222423942D
:2061C000312C8090BA059090BB05092C000CAA08BB08E091B805F091B905E20DF31DEE0F94
:2061E000FF1FEA55FF4F20813181032E000C440B550B281939094A095B09A1E1BFEF0E94A9
:206200008E362091BC053091BD05032E000C440B550B281939094A095B090E9461362151F4
:206220003F4F4F4F5F4F5901203F31051CF03FEEA32EB12CB7FE02C0B12CA12CF301F18127
:20624000FC8321012AE0420E511C410139E0830E911C8F2F90E0412F50E0F12CE12C8C01B8
:206260009201B40188E297E00E94B50D20EEE22E27E0F22E85019201A601B40188E297E0F6
:206280000E94B50DF301A182FFEF2F1A3F0A2FEF621A720A1C8165013CE2231631E0330649
:2062A00009F08FCF4CCA8091F2068D3009F482CE8091F2068B3009F0BEC01091BE05C0906F
:2062C000BA05D090BB050D2C000CEE08FF08E091B805F091B905EE0FFF1FEA57FE4F2081E6
:2062E0003181032E000C440B550B2C193D094E095F09A1E1BFEF0E948E362091BC053091ED
:20630000BD05032E000C440B550B2C193D094E095F090E94613669017A016FEEC60ED11C49
:20632000E11CF11C80EFC816D1041CF06FEEC62ED12CD7FE02C0D12CC12CC092BE05EEEB68
:20634000F5E0FD83EC834AE0642E712C22242394312C8090BA059090BB05092C000CAA0824
:20636000BB08E091B805F091B905E20DF31DEE0FFF1FE857FE4F20813181032E000C440B68
:20638000550B281939094A095B09A1E1BFEF0E948E362091BC053091BD05032E000C440B4C
:2063A000550B281939094A095B090E94613621513F4F4F4F5F4F5901203F31051CF02FEEA6
:2063C000A22EB12CB7FE02C0B12CA12CEC81FD8191802301F4E04F0E511C892D90E0412F9B
:2063E00050E0F12CE12C8C019201B30188E297E00E94B50D90EEE92E97E0F92E85019201DE
:20640000A601B30188E297E00E94B50DEC81FD81A182FFEF2F1A3F0A2C813D812F5F3F4FC7
:206420003D832C83192D650132013BE42316310409F08FCF84C98091F2068E3009F43DCF0D
:206440008091F2068F3009F478C98091F206803109F473C98091F206813109F070C96DC920
:2064600082E082C980910907811103C084E090E190C981E090E18DC989E1B8C987E091E0E0
:20648000BEC9072E000C880B990B0E94173824EC3AEB4AE85BE3E2C989EF9FE00E94120D04
:2064A0008091FE066091FC067091FD06813069F4072E000C880B990B0E94173826ED3CE02A
:2064C0004FE15DE30E94CC38D1C9072E000C880B990B0E94173823EF3DEE47E95BE3F2CF37
:2064E00087E091E0F0C9072E000C880B990B0E94173824EC3AEB4AE85BE30ECA87E091E04D
:206500002ACA072E000C880B990B0E94173824EC3AEB4AE85BE348CA10923B0710923A07A0
:20652000109239071092380783EE90E0909335078093340788E390E090933707809336077E
:2065400089EE9FE00E94120D47E050E068E370E083EE90E00E94CF158FEF97E090933B07D1
:2065600080933A079093390780933807C090F706D090F806E090F906F090FA0624EF3DEF39
:206580004FE151E4C701B6010E94683787FF43C043E050E0C701B6010E947E1A86EE9FE04E
:2065A0000E94120D45E050E06AE470E08BEF90E00E94CF158FEF97E090933B0780933A0709
:2065C0009093390780933807C090F306D090F406E090F506F090F60625E83BEE4FE151E4E1
:2065E000C701B6010E94683742E050E087FD0CC026E636EE47EC52E4C701B6010E946837E0
:2066000087FF68C041E050E0C701B6010E947E1A8DEC9FE001CA21E73DEF47EC52E4C7019A
:20662000B6010E94683787FF09C042E050E0C701B6010E947E1A83EE9FE0B2CF2DEC3CEF53
:2066400049E754E4C701B6010E94683787FF09C041E050E0C701B6010E947E1A80EE9FE0CC
:206660009FCF20E030E04AE754E4C701B6010E946D374B015C0120E03CE24CE156E4C70178
:20668000B6010E94683787FF09C042E050E0C501B4010E947E1A8CED9FE082CF20E037E349
:2066A00043EC57E4C701B6010E94683787FF09C041E050E0C501B4010E947E1A88ED9FE067
:2066C0006FCF50E040E0C501B4010E947E1A84ED9FE066CF8FEC9FE00E94120D99CF20917E
:2066E00007070CE017E028301CF421E043E0E9C922E044E0E6C9209107070CE017E028309C
:2067000014F421E002CA22E000CA209107070CE017E0283014F421E017CA22E044E00E942C
:20672000EF338091090718160CF011CA80910E0780930D0780910F0780930E07809110074D
:2067400080930F07809111078093100700CA0E94321F0E94FA160AE010E080910A078823A7
:20676000A1F180910C01181614F40E940E1680910907181614F588E00E94AE08892BB9F4F4
:20678000209107078091050790910607B8010E9499392530ACF070930407609303070E9424
:2067A000321F1092080710920A070E940E166AE070E080E090E00E9481090E94FA16CDCF7A
:2067C0007093020760930107EACF80E090E0892B11F40C9480280E9400000C948028EF92BD
:2067E0000F931F93CF93DF93E80134E047FD34E1042E000C550B57FF03C05195419551094E
:20680000E32E022F242FAE010E941434CE01DF91CF911F910F91EF900895FB01DC010590D1
:206820000D920020E1F70895A9E0B0E0EAE1F4E30C9499366A01F22EB02E102FFBE3AF2E97
:20684000A01608F41BE31F5F012F27E0AE014F5F5F4F0E947335BC018981982F9970913026
:2068600009F43FC09BE2E1FC04C09E2D9170E0FC3AC05E2D5071E82FE87083FF46C084E0B5
:20688000911101C083E0EF2DE81B8F1508F0E0E0D6018E2F20E2552351F1992329F0D601BB
:2068A0009C93C60101966C0196012D5F3F4FE2FE24C08EE4D6018C9391E411969C9311970E
:2068C00012968C93D9018E2F90E281111BC0E20FF32FF11D10828EEF9FEF2996ECE00C9492
:2068E000B5369DE2C6CF90E2C4CF2D9381508111FCCFCE0ED11CE0E0D0CF8EE6D6018C9314
:2069000091E6DBCF9D938150E0CF482F447082FF3DC084E0911101C083E08F1510F4EF2D0F
:20692000E81BD6018E2F20E2552309F1992329F0D6019C93C60101966C0196012D5F3F4FF5
:20694000E2FE1BC089E4D6018C938EE411968C93119786E412968C93D9018E2F90E2882354
:2069600009F4B5CF9D938150FACF2D9381508111FCCFCE0ED11CE0E0D9CF89E6D6018C9348
:206980008EE611968C93119786E6E4CF9B0177FF02C030E020E0A1E0B0E0911102C0B0E00D
:2069A000A0E0F9013196AE0FBF1F8B2C912CBB2009F461C05401EFEFAE1ABE0AAA0DBB1D3C
:2069C000FA161B0619F014F04F2D4A1B511188C0E3FC59C07601A42FB0E2A1114FC0C40E87
:2069E000D11C992309F45BC040E0D6011196F60190836D01552309F448C0012F060F9A81E3
:206A0000582F507184FF03C0913309F4015010160CF047C0093008F008E0EEE2FE2E5B013C
:206A2000A01AB10885019194819491082F3F320729F4D601FC92F60131966F016217730740
:206A400094F1021713077CF5DB01A21BB30BAA24A394B12CAC0EBD1EAA0DBB1D11968C91EC
:206A600021503109D601119628153905F4F0F60180836D01DBCFB12CA12CA0CFF701B19327
:206A80007F01A150AACF9111B0CFD601942F50E302C05D9391509111FCCFC40ED11C40E03F
:206AA000ACCF01E0BACF80E3DBCF6217730731F4963388F4953311F4552369F0F6018083EF
:206AC000FD01842F90E2811108C0A40FB11D1C9290E080E002CF81E3F1CF91938150F3CF8E
:206AE000911183CF8ACF283008F027E03327DA01990F311D87FD916000966105710539F4B3
:206B000032602E5F3D9330E32A95E1F708959F3F30F080387105610509F03C5F3C5F3D93AE
:206B2000913008F08068911DDF93CF931F930F93FF92EF92192F987F9695E92F96959695D4
:206B4000E90FFF27EE53FF4F99273327EE24FF24A701E70105900894079428F4360FE71E77
:206B6000F81E491F511D660F771F881F991F0694A1F70590079428F4E70EF81E491F561F59
:206B8000C11D770F881F991F661F0694A1F70590079428F4F80E491F561FC71FD11D880FE1
:206BA000991F661F771F0694A1F70590079420F4490F561FC71FD81F990F661F771F881F78
:206BC0000694A9F784911095177041F0D695C79557954795F794E7941A95C1F7E8E6F0E06F
:206BE00068941590159135916591959105907FE27395E118F10A430B560BC90BD009C0F767
:206C0000E10CF11E431F561FC91FD01D7EF4703311F48A95E6CFE894015030F0080F0AF4DC
:206C20000027021708F4202F2395022F7A3328F079E37D932A95E9F710C07D932A9589F6F2
:206C4000069497956795379517951794E118F10A430B560BC90BD00998F023957E917395A8
:206C60007A3308F070E37C932013B8F77E9170617D9330F0839571E37D9370E32A95E1F7B5
:206C80001124EF90FF900F911F91CF91DF91992787FD90950895F999FECF92BD81BDF89A0D
:206CA000992780B50895262FF999FECF1FBA92BD81BD20BD0FB6F894FA9AF99A0FBE01966F
:206CC0000895052E97FB1EF400940E94783657FD07D00E94CA3607FC03D04EF40C94783629
:206CE00050954095309521953F4F4F4F5F4F089590958095709561957F4F8F4F9F4F08957C
:206D00000E94EC36A59F900DB49F900DA49F800D911D11240895B7FF0C9480360E9480362A
:206D2000821B930B08952F923F924F925F926F927F928F929F92AF92BF92CF92DF92EF92CE
:206D4000FF920F931F93CF93DF93CDB7DEB7CA1BDB0B0FB6F894DEBF0FBECDBF09942A8800
:206D6000398848885F846E847D848C849B84AA84B984C884DF80EE80FD800C811B81AA8128
:206D8000B981CE0FD11D0FB6F894DEBF0FBECDBFED010895A1E21A2EAA1BBB1BFD010DC0EB
:206DA000AA1FBB1FEE1FFF1FA217B307E407F50720F0A21BB30BE40BF50B661F771F881F6F
:206DC000991F1A9469F760957095809590959B01AC01BD01CF010895A29FB001B39FC00140
:206DE000A39F700D811D1124911DB29F700D811D1124911D08955058BB27AA270E94133720
:206E00000C948D380E947F3838F00E94863820F039F49F3F19F426F40C947C380EF4E0951F
:206E2000E7FB0C947638E92F0E949E3858F3BA17620773078407950720F079F4A6F50C94B4
:206E4000C0380EF4E0950B2EBA2FA02D0B01B90190010C01CA01A0011124FF27591B99F0AC
:206E6000593F50F4503E68F11A16F040A22F232F342F4427585FF3CF469537952795A795E6
:206E8000F0405395C9F77EF41F16BA0B620B730B840BBAF09150A1F0FF0FBB1F661F771F15
:206EA000881FC2F70EC0BA0F621F731F841F48F4879577956795B795F7959E3F08F0B0CF99
:206EC0009395880F08F09927EE0F9795879508950E94523808F481E008950E9481370C9439
:206EE0008D380E94863858F00E947F3840F029F45F3F29F00C94763851110C94C1380C94DF
:206F00007C380E949E3868F39923B1F3552391F3951B550BBB27AA2762177307840738F025
:206F20009F5F5F4F220F331F441FAA1FA9F335D00E2E3AF0E0E832D091505040E695001C1D
:206F4000CAF72BD0FE2F29D0660F771F881FBB1F261737074807AB07B0E809F0BB0B802D43
:206F6000BF01FF2793585F4F3AF09E3F510578F00C9476380C94C1385F3FE4F3983ED4F3D4
:206F8000869577956795B795F7959F5FC9F7880F911D9695879597F90895E1E0660F771FB3
:206FA000881FBB1F621773078407BA0720F0621B730B840BBA0BEE1F88F7E09508950E9472
:206FC000E6376894B1110C94C13808950E94A63888F09F5798F0B92F9927B751B0F0E1F009
:206FE000660F771F881F991F1AF0BA95C9F714C0B13091F00E94C038B1E008950C94C03878
:20700000672F782F8827B85F39F0B93FCCF3869577956795B395D9F73EF4909580957095E1
:2070200061957F4F8F4F9F4F0895E89409C097FB3EF490958095709561957F4F8F4F9F4F4B
:207040009923A9F0F92F96E9BB279395F695879577956795B795F111F8CFFAF4BB0F11F4A9
:2070600060FF1BC06F5F7F4F8F4F9F4F16C0882311F096E911C0772321F09EE8872F762F10
:2070800005C0662371F096E8862F70E060E02AF09A95660F771F881FDAF7880F96958795D4
:2070A00097F90895990F0008550FAA0BE0E8FEEF16161706E807F907C0F012161306E40711
:2070C000F50798F0621B730B840B950B39F40A2661F0232B242B252B21F408950A2609F488
:2070E000A140A6958FEF811D811D089597F99F6780E870E060E008959FEF80EC0895002437
:207100000A941616170618060906089500240A9412161306140605060895092E0394000C1F
:2071200011F4882352F0BB0F40F4BF2B11F460FF04C06F5F7F4F8F4F9F4F089557FD90580C
:20714000440F551F59F05F3F71F04795880F97FB991F61F09F3F79F08795089512161306D1
:207160001406551FF2CF4695F1DF08C0161617061806991FF1CF869571056105089408953E
:20718000E894BB2766277727CB0197F908950E94523808F48FEF08950E94DF380C948D380C
:2071A0000E947F3838F00E94863820F0952311F00C9476380C947C3811240C94C1380E9413
:2071C0009E3870F3959FC1F3950F50E0551F629FF001729FBB27F00DB11D639FAA27F00DC6
:2071E000B11DAA1F649F6627B00DA11D661F829F2227B00DA11D621F739FB00DA11D621FF4
:20720000839FA00D611D221F749F3327A00D611D231F849F600D211D822F762F6A2F112414
:207220009F5750409AF0F1F088234AF0EE0FFF1FBB1F661F771F881F91505040A9F79E3FD3
:20724000510580F00C9476380C94C1385F3FE4F3983ED4F3869577956795B795F795E795F8
:207260009F5FC1F7FE2B880F911D9695879597F9089519F416F40C947C380C9484390E940C
:20728000A638B8F39923C9F3B6F39F57550B87FF0E9492390024A0E640EA900180585695D3
:2072A000979528F4805C660F771F881F20F026173707480730F4621B730B840B20293129CD
:2072C0004A2BA69517940794202531254A2758F7660F771F881F20F026173707480730F4AD
:2072E000620B730B840B200D311D411DA09581F7B901842F9158880F9695879508950E941B
:207300005238880B990B08959F3F31F0915020F4879577956795B795880F911D969587951F
:2073200097F9089591505040660F771F881FD2F7089597FB072E16F4009407D077FD09D00E
:207340000E94C23907FC05D03EF4909581959F4F0895709561957F4F0895EE0FFF1F0590AA
:20736000F491E02D09940E94EC36332312F48A1B9B0B0C94BD390E94EC36B7FF0895821B29
:20738000930B0895AA1BBB1B51E107C0AA1FBB1FA617B70710F0A61BB70B881F991F5A952F
:2073A000A9F780959095BC01CD01089581E090E0F8940C94DB39F894FFCF01787878417343
:2073C00000787878780002FF835700000000400C5808CC15CB154713DB09290F010F1D0FD3
:2073E000110F300FDB0982139211891976198512DD16B50D560D0D0A006E616E00696E66A1
:20740000006F76660000FFFFFFFFFFFFFFFFFFFFFFFFFFFFFFFFFFFFFFFFFFFFFFFFFFFF3B
:20742000FFFFFFFFFFFFFFFFFFFFFFFFFFFFFFFFFFFFFFFFFFFFFFFFFFFFFFFFFFFFFFFF6C
:20744000FFFFFFFFFFFFFFFFFFFFFFFFFFFFFFFFFFFFFFFFFFFFFFFFFFFFFFFFFFFFFFFF4C
:20746000FFFFFFFFFFFFFFFFFFFFFFFFFFFFFFFFFFFFFFFFFFFFFFFFFFFFFFFFFFFFFFFF2C
:20748000FFFFFFFFFFFFFFFFFFFFFFFFFFFFFFFFFFFFFFFFFFFFFFFFFFFFFFFFFFFFFFFF0C
:207E0000112484B714BE81FFF0D085E08093810082E08093C00088E18093C10086E08093FC
:207E2000C20080E18093C4008EE0C9D0259A86E020E33CEF91E0309385002093840096BBAD
:207E4000B09BFECF1D9AA8958150A9F7CC24DD2488248394B5E0AB2EA1E19A2EF3E0BF2E79
:207E6000A2D0813461F49FD0082FAFD0023811F0013811F484E001C083E08DD089C0823404
:207E800011F484E103C0853419F485E0A6D080C0853579F488D0E82EFF2485D0082F10E0A0
:207EA000102F00270E291F29000F111F8ED068016FC0863521F484E090D080E0DECF84364D
:207EC00009F040C070D06FD0082F6DD080E0C81680E7D80618F4F601B7BEE895C0E0D1E0ED
:207EE00062D089930C17E1F7F0E0CF16F0E7DF0618F0F601B7BEE89568D007B600FCFDCF1A
:207F0000A601A0E0B1E02C9130E011968C91119790E0982F8827822B932B1296FA010C016F
:207F200087BEE89511244E5F5F4FF1E0A038BF0751F7F601A7BEE89507B600FCFDCF97BE85
:207F4000E89526C08437B1F42ED02DD0F82E2BD03CD0F601EF2C8F010F5F1F4F84911BD0B8
:207F6000EA94F801C1F70894C11CD11CFA94CF0CD11C0EC0853739F428D08EE10CD085E9AE
:207F80000AD08FE07ACF813511F488E018D01DD080E101D065CF982F8091C00085FFFCCF0A
:207FA0009093C60008958091C00087FFFCCF8091C00084FD01C0A8958091C6000895E0E68F
:207FC000F0E098E1908380830895EDDF803219F088E0F5DFFFCF84E1DECF1F93182FE3DF47
:207FE0001150E9F7F2DF1F91089580E0E8DFEE27FF270994FFFFFFFFFFFFFFFFFFFF040425
:00000001FF
